:100000000C942A001895000018950000189500001F
:10001000189500001895000018950000189500002C
:100020001895000018950000189500000C94C40164
:10003000189500000C94440F0C94760F189500004E
:1000400018950000189500001895000018950000FC
:10005000189500008FE58DBFCCEFECE44E2E88E0C4
:100060008EBFD7E0F7E05F2EEEEFF7E0A0E6B0E05E
:10007000A89584B7082E877F84BF88E1992781BD22
:1000800091BD88278D933197E9F780E189B980E0A8
:1000900080BD88E18AB96624579A0E94591084B7B6
:1000A000877F84BF88E181BD80E081BD80E08ABB1D
:1000B0008CE187BB83EE88BB80E084BB8FEF85BB80
:1000C00080EF81BB8FE082BB87E886B980E087B98B
:1000D000379A85E083BF81EB8FBD81E08EBD8FEFC6
:1000E0008ABDA0EAB1E0ECEBF0E20E94900DA2EA3A
:1000F000B1E0EEEBF0E20E94900D8FEF8ABD80E060
:1001000088BD0CEF13E020E030E0ABECB0E00D93E5
:100110001D932D933C9380E08093FB00C29A86E967
:1001200090E00E945E0DC39A86E990E00E945E0D09
:10013000C49A8AEF90E00E945E0DC298C398C4985A
:1001400080E090E0A1ECB0E08D939C9301E010E0A2
:1001500020E030E0A7EDB0E00D931D932D933C938C
:100160004AE050E060E070E0A7EDB0E00D911D9135
:100170002D913C910E94A70F1CF011F00C94E0000F
:10018000A1ECB0E00D911C910F931F9307B1007E7D
:10019000076007B90E94960D482F592F1F910F91A4
:1001A000040F151FA1ECB0E00D931C9381E090E0CB
:1001B0000E945E0DA7EDB0E00E940D0C0C94B00003
:1001C000A1ECB0E00D911C914AE050E00E942D0C92
:1001D000A1ECB0E04D935C9382E090E00E945E0D54
:1001E000A1ECB0E00D911C91043650E015070CF421
:1001F00002C00C94000184E0809310010C949609D5
:100200000E942108789489B7816089BFE0ECF0E210
:100210000E94BB0CE6ECF0E20E94BB0C0E94C20CF8
:1002200000919601013011F00C94440180E080931C
:100230009601A1E1B1E03FE30E94760CA1E1B1E0BB
:100240008C91082F0A3011F00C944201A1E1B1E029
:100250000E945310082F41E0041BA7E9B1E00C9362
:10026000A1E1B1E00E945310EA2FFB2F009197010A
:100270003197E01BF10B0FEFA1E1B1E00E944B10B1
:100280000C941E010E94D20988E090E00E945E0D4D
:10029000EEECF0E20E94BB0CA4E3B7E0EFEDF0E07F
:1002A0000E94BD0F0E94B30C0E94C20C88E090E037
:1002B0000E945E0DE4EDF0E20E94BB0CA4E3B7E007
:1002C000EBEEF0E00E94BD0F0E94B30C0E94C20C46
:1002D00088E090E00E945E0DEAEDF0E20E94BB0C27
:1002E000A4E3B7E0E7EFF0E00E94BD0F0E94B30C7B
:1002F0000E94C20C88E090E00E945E0DE0EEF0E209
:100300000E94BB0CA4E3B7E0ECEFF0E00E94BD0F4D
:100310000E94B30C0E94C20C88E090E00E945E0D27
:10032000E6EEF0E20E94BB0CA4E3B7E0E7EEF0E0FB
:100330000E94BD0F0E94B30C0E94C20C88E090E0A6
:100340000E945E0DECEEF0E20E94BB0CA4E3B7E06D
:10035000E3EEF0E00E94C20F0E94B30C0E94C20CB8
:1003600088E090E00E945E0DE2EFF0E20E94BB0C9C
:10037000A4E3B7E0E5EEF0E00E94C20F0E94B30CE8
:100380000E94C20C0C9410010F921F922F923F9268
:100390004F925F927F92AF92BF920F931F932F93D2
:1003A0003F934F935F936F937F938F939F93AF93FD
:1003B000BF93CF93DF93EF93FF938FB78F93A8955E
:1003C00084E6809352000E940B020E94AC030E94BC
:1003D00069040E949C050E94BE060E9494078F91AA
:1003E0008FBFFF91EF91DF91CF91BF91AF919F911F
:1003F0008F917F916F915F914F913F912F911F91BD
:100400000F91BF90AF907F905F904F903F902F9053
:100410001F900F90189507B1007E056007B90E94E4
:10042000960DABEBB0E08D939D9388278D938C93C5
:1004300000E014E020E030E0ABEBB0E04D915D91E6
:100440006D917C910E94A20FABEBB0E00D931D93D8
:100450002D933D9307B1007E036007B90E94960D6E
:10046000A7EBB0E08D939D9388278D938C9307B174
:10047000007E006007B90E94960DAFEBB0E08D934F
:100480009C9307B1007E066007B90E94960DA0E01C
:10049000B1E08D939C9300E014E00F931F9307B19C
:1004A000007E076007B90E94960D482F592F1F91B3
:1004B0000F91041B150BA1ECB0E00D931C93A7EB5F
:1004C000B0E00D911D912D913C914AE050E060E02B
:1004D00070E00E946D0DA7EBB0E00D931D932D937E
:1004E0003D93ABEBB0E00D911D912D913C914AE015
:1004F00050E060E070E00E946D0DABEBB0E00D935A
:100500001D932D933D93A3ECB0E00D911D912D9182
:100510003C9146E950E060E070E00E94F60CA7EDE7
:10052000B0E04D935D936D937D93A3ECB0E00D919E
:100530001D912D913C91A7EDB0E04D915D916D9194
:100540007C910E94A20FA3ECB0E00D931D932D931C
:100550003D93A7EBB0E00D911D912D913C91ACE046
:10056000B1E04D915C91662777270E94A20FA7ED1D
:10057000B0E00D931D932D933D93A3ECB0E00D914E
:100580001D912D913C91A7EDB0E04D915D916D9144
:100590007C910E949D0FA3ECB0E00D931D932D93D1
:1005A0003D93A7ECB0E00D911D912D913C9146E952
:1005B00050E060E070E00E94F60CA3EDB0E04D93D7
:1005C0005D936D937D93A7ECB0E00D911D912D91FE
:1005D0003C91A3EDB0E04D915D916D917C910E94B5
:1005E000A20FA7ECB0E00D931D932D933D93A7ECC4
:1005F000B0E00D911D912D913C91ABEBB0E04D9190
:100600005D916D917C910E949D0FA7ECB0E00D93E0
:100610001D932D933D93A7ECB0E00D911D912D916D
:100620003C914FE050E060E070E00E94F60CA3EDDA
:10063000B0E04D935D936D937D93ABEBB0E00D9186
:100640001D912D913C914AE050E060E070E00E94E5
:100650006D0DA7EDB0E00D931D932D933D93A3ED8C
:10066000B0E00D911D912D913C91A7EDB0E04D9121
:100670005D916D917C910E94A20FA3EDB0E00D936E
:100680001D932D933D93A3EDB0E00D911D912D9100
:100690003C914EE150E060E070E00E946D0DA3EDF2
:1006A000B0E00D931D932D933D93A3EDB0E00D911C
:1006B0001D912D913C9144E650E060E070E00E9475
:1006C000F60CA3EFB0E04D935D936D937D93A3EC97
:1006D000B0E00D911D912D913C91A3EFB0E04D91B3
:1006E0005D916D917C910E949D0FA3ECB0E00D9304
:1006F0001D932D933D9306E910E020E030E0A7ED37
:10070000B0E00D931D932D933C93A3ECB0E00D91BD
:100710001D912D913C91A7EDB0E04D915D916D91B2
:100720007C910E94F60CAFEDB0E04D935D936D931C
:100730007D93A3EFB0E00D911D912D913C914AE086
:1007400050E060E070E00E94F60CA3EFB0E04D9343
:100750005D936D937D930895AFEDB0E00D911D9184
:100760002D913C91AFEEB0E04D915D916D917C91FA
:100770000E949D0FA7EFB0E00D931D932D933D9325
:10078000A3EFB0E00D911D912D913C91A7EFB0E04A
:100790004D915D916D917C910E949D0FA7EFB0E00E
:1007A0000D931D932D933D93A7EFB0E00D911D91F7
:1007B0002D913C9141E150E060E070E00E946D0DB0
:1007C000A7EFB0E00D931D932D933D93ACEFB0E0F8
:1007D0000D911D912D913C91A7EFB0E04D915D9150
:1007E0006D917C910E949D0FACEFB0E00D931D9335
:1007F0002D933D9348ED56ED60E070E0ACEFB0E036
:100800000D911D912D913C910E94A70F1CF011F0AC
:100810000C940C040C94160408ED16ED20E030E066
:10082000ACEFB0E00D931D932D933C9348E259E259
:100830006FEF7FEFACEFB0E00D911D912D913C91EA
:100840000E94A70F0CF402C00C94300408E219E2D5
:100850002FEF3FEFACEFB0E00D931D932D933C9342
:10086000ACEFB0E00D911D912D913C914BE950E022
:1008700060E070E00E94F60CA7EDB0E04D935D9350
:100880006D937D93A7EFB0E00D911D912D913C915B
:1008900045EA50E060E070E00E94F60CA3EDB0E0A5
:1008A0004D935D936D937D93A7EDB0E00D911D91F8
:1008B0002D913C91A3EDB0E04D915D916D917C91B6
:1008C0000E949D0FA7EEB0E00D931D932D933D93D5
:1008D0000895AAE0B1E00D911D9117FB1EF42FEFD2
:1008E0003FEF02C022273327A0E0B1E04D915D9198
:1008F00057FB1EF46FEF7FEF02C0662777270E9439
:10090000A20FA6E0B1E00D931D932D933D93ACEFA4
:10091000B0E00D911D912D913C9140E25EE460E0CC
:1009200070E00E94F60CA3EDB0E04D935D936D93E3
:100930007D93A3EDB0E00D911D912D913C910E940E
:100940004A0DA3EDB0E00D931D932D933D9342E02E
:1009500050E060E070E0A3EDB0E00D911D912D91AD
:100960003C910E94A70F0CF402C00C94C10402E059
:1009700010E020E030E0A3EDB0E00D931D932D9347
:100980003C93A6E0B1E00D911D912D913C91A3ED1A
:10099000B0E04D915D916D917C910E94F60CA6E0C6
:1009A000B1E04D935D936D937D93ACEFB0E00D910D
:1009B0001D912D913C9140ED57E060E070E00E9468
:1009C000F60CA3EDB0E04D935D936D937D93A3ED95
:1009D000B0E00D911D912D913C910E944A0DA3ED27
:1009E000B0E00D931D932D933D9346E150E060E000
:1009F00070E0A3EDB0E00D911D912D913C910E940E
:100A0000A70F1CF011F00C9407050C94110506E1DA
:100A100010E020E030E0A3EDB0E00D931D932D93A6
:100A20003C930BE110E020E030E0A3EDB0E04D910D
:100A30005D916D917C910E94A20FA3EDB0E00D93AA
:100A40001D932D933D93A3EDB0E00D911D912D913C
:100A50003C914FEF5FEF6FEF7FEF0E946D0DABEDBD
:100A6000B0E00D931D932D933D93A3EDB0E04D9118
:100A70005D916D917C91A6E0B1E00D911D912D915C
:100A80003C910E94A70F1CF011F00C9449050C94A6
:100A90005505A3EDB0E00D911D912D913C91A6E07F
:100AA000B1E00D931D932D933C93ABEDB0E04D91D0
:100AB0005D916D917C91A6E0B1E00D911D912D911C
:100AC0003C910E94A70F0CF402C00C947305ABED8F
:100AD000B0E00D911D912D913C91A6E0B1E00D93F8
:100AE0001D932D933C93A6E0B1E00D911D912D91A6
:100AF0003C91ABEEB0E00D931D932D933C93A7EE8C
:100B0000B0E00D911C91ABEEB0E04D915C91041BF7
:100B1000150BA3EEB0E00D931C93A7EEB0E00D9182
:100B20001C91ABEEB0E04D915C91040F151FA5EE4A
:100B3000B0E00D931C9308950091FB00003011F07C
:100B40000C94080680E090E0A3EEB0E08D939C93B7
:100B500080E090E0A5EEB0E08D939C9300E010E083
:100B600020E030E0A7EEB0E00D931D932D933C9371
:100B700000E010E020E030E0AFEEB0E00D931D9318
:100B80002D933C9300E010E020E030E0ACEFB0E0CB
:100B90000D931D932D933C9300E010E020E030E096
:100BA000AFEDB0E00D931D932D933C9300E010E06A
:100BB00020E030E0A3ECB0E00D931D932D933C9327
:100BC00000E010E020E030E0A2E0B1E00D931D93E2
:100BD0002D933C93A1ECB0E00D911C91023350E0B9
:100BE00015071CF011F00C94F7050C9406060E94F2
:100BF000210881E08093FB0000E010E020E030E07D
:100C0000A2E0B1E00D931D932D933C930C94BD068F
:100C1000013011F00C941C06A1ECB0E00D911C9178
:100C2000023350E015070CF402C00C941A0683E05E
:100C30008093FB000C94BD06033011F00C94BA06AF
:100C400081B5886181BD877F81BD00E010E020E033
:100C500030E0A2E0B1E00D931D932D933C9301E0B1
:100C600010E020E030E0A3EDB0E00D931D932D9354
:100C70003C934FEF50E060E070E0A3EDB0E00D91E9
:100C80001D912D913C910E94A70F1CF011F00C9426
:100C9000B206A3EEB0E00D911C91003050E01507B4
:100CA00081E009F080E08F93A5EEB0E00D911C91FA
:100CB000003050E0150781E009F080E09F91892322
:100CC000882311F40C9466060C94B206A3EEB0E0EF
:100CD0000D911C91003050E015071CF011F00C94A0
:100CE00073060C947706A3EEB0E00E94230CA3EEEB
:100CF000B0E00D911C91003050E015070CF402C0DB
:100D00000C948606A3EEB0E00E941C0CA5EEB0E0A9
:100D10000D911C91003050E015071CF011F00C945F
:100D200093060C949706A5EEB0E00E94230CA5EE66
:100D3000B0E00D911C91003050E015070CF402C09A
:100D40000C94A606A5EEB0E00E941C0C89E190E090
:100D50000E945E0D0E94BE06A3EDB0E00E940D0C45
:100D60000C94390680E08093FB0081B5886081BDDA
:100D70000C94BD0683E08093FB000895A3EEB0E0E1
:100D80000D911C91043B50E015071CF011F00C94E0
:100D9000CB060C94D30684EB90E0A3EEB0E08D93E9
:100DA0009C930C94E406A3EEB0E00D911C910C34DE
:100DB0005FEF15070CF402C00C94E4068CE49FEF7F
:100DC000A3EEB0E08D939C93A5EEB0E00D911C9145
:100DD000043B50E015071CF011F00C94F1060C9444
:100DE000F90684EB90E0A5EEB0E08D939C930C9413
:100DF0000A07A5EEB0E00D911C910C345FEF1507CA
:100E00000CF402C00C940A078CE49FEFA5EEB0E04E
:100E10008D939C93A2E3B0E08C9186FBA6EBB0E0AF
:100E20008C9185F98C93A2E3B0E08C9187FBA6EBC3
:100E3000B0E08C9184F98C93A3EEB0E00D911C91FD
:100E4000003050E015070CF402C00C942A07969A63
:100E50000C942B079698A5EEB0E00D911C910030F4
:100E600050E015070CF402C00C943907979A0C94C3
:100E70003A0797980027A6EBB0E08C9185FB0EF41B
:100E800001E04427A2E3B0E08C9186FB0EF4439589
:100E9000041711F40C9453078091B6008068809376
:100EA000B6000C9458078091B6008F778093B600F7
:100EB0000027A6EBB0E08C9184FB0EF401E0442700
:100EC000A2E3B0E08C9187FB0EF44395041711F474
:100ED0000C9471078091B60080648093B6000C94E6
:100EE00076078091B6008F7B8093B600A3EEB0E0CA
:100EF0008D919C910E944D0CAFECB0E08D939C9332
:100F0000A5EEB0E08D919C910E944D0CA1EDB0E05A
:100F10008D939C930FEF4091CF00041B0ABDA1ED70
:100F2000B0E08C9188BD0895ABECB0E00D911D91BF
:100F30002D913C914CE251E060E070E00E94F60C93
:100F4000A3EDB0E04D935D936D937D93ABECB0E07A
:100F50000D911D912D913C91A3EDB0E04D915D91CE
:100F60006D917C910E94A20FABECB0E00D931D93AC
:100F70002D933D93ABECB0E00D911D912D913C91E3
:100F8000AFEBB0E04D915D9157FB1EF46FEF7FEF3B
:100F900002C0662777270E949D0FABECB0E00D934F
:100FA0001D932D933D93ABECB0E00D911D912D91D0
:100FB0003C914CE251E060E070E00E94F60CA3ED41
:100FC000B0E04D935D936D937D934CEF53E060E003
:100FD00070E0A3EDB0E00D911D912D913C910E9428
:100FE000A70F1CF011F00C94F7070C94FA07C29AA3
:100FF000C398C4984CEF53E060E070E0A3EDB0E01C
:101000000D911D912D913C910E94A70F0CF402C0EF
:101010000C940D08C39AC498C29840EC53E060E069
:1010200070E0A3EDB0E00D911D912D913C910E94D7
:10103000A70F0CF402C00C942008C398C298C49A5D
:10104000089581B5886181BD877F81BD80E090E092
:10105000A0E0B1E08D939C9301E010E020E030E04F
:10106000A7EDB0E00D931D932D933C934AE050E023
:1010700060E070E0A7EDB0E00D911D912D913C91E5
:101080000E94A70F1CF011F00C946608A0E0B1E0DC
:101090000D911C910F931F9307B1007E066007B955
:1010A0000E94960D482F592F1F910F91040F151F65
:1010B000A0E0B1E00D931C9381E090E00E945E0DF2
:1010C000A7EDB0E00E940D0C0C943608A0E0B1E052
:1010D0000D911C914AE050E00E942D0CAAE0B1E075
:1010E0004D935C9300E010E020E030E0ABEBB0E02B
:1010F0000D931D932D933C9301E010E020E030E030
:10110000A7EDB0E00D931D932D933C9346E950E07D
:1011100060E070E0A7EDB0E00D911D912D913C9144
:101120000E94A70F1CF011F00C94E50807B1007E97
:10113000056007B90E94960DA3EDB0E08D939D93D5
:1011400088278D938C9300E014E020E030E0A3ED3D
:10115000B0E04D915D916D917C910E94A20FA3ED45
:10116000B0E00D931D932D933D93A3EDB0E00D9151
:101170001D912D913C914AE050E060E070E00E94AA
:101180006D0DA3EDB0E00D931D932D933D93ABEB4F
:10119000B0E00D911D912D913C91A3EDB0E04D91EA
:1011A0005D916D917C910E949D0FABEBB0E00D9332
:1011B0001D932D933D9382E090E00E945E0DA7ED7C
:1011C000B0E00E940D0C0C948608ABEBB0E00D91E2
:1011D0001C9146E950E00E94530CAEE0B1E04D9303
:1011E0005C93ABEBB0E00D911D912D913C91A7EC80
:1011F000B0E00D931D932D933C9300E010E020E0B0
:1012000030E0A7EBB0E00D931D932D933C9301E0EC
:1012100010E020E030E0A7EDB0E00D931D932D939A
:101220003C9344E650E060E070E0A7EDB0E00D9143
:101230001D912D913C910E94A70F1CF011F00C9470
:101240004C0907B1007E036007B90E94960DA3ED1B
:10125000B0E08D939D9388278D938C93A7EBB0E09E
:101260000D911D912D913C91A3EDB0E04D915D91BB
:101270006D917C910E949D0FA7EBB0E00D931D93A3
:101280002D933D9382E090E00E945E0DA7EDB0E0CB
:101290000E940D0C0C941109A7EBB0E00D911C916C
:1012A0004AE050E00E94530CACE0B1E04D935C93F7
:1012B00081B5886081BDACE0B1E00D911C91003A30
:1012C0005FE0150710F00C94680983E0809310012B
:1012D000ACE0B1E00D911C91003757E1150718F013
:1012E00011F00C9475090C94780983E08093100137
:1012F000AEE0B1E00D911C91063950E0150710F0F9
:101300000C94850982E080931001AEE0B1E00D916C
:101310001C910C3251E0150718F011F00C94920951
:101320000C94950982E080931001089581B588613D
:1013300081BD877F81BD01E010E020E030E0A7EDB6
:10134000B0E00D931D932D933C93A0E1B1E04C913F
:10135000552766277727A7EDB0E00D911D912D91B8
:101360003C910E94A70F1CF011F00C94C709C49A7D
:1013700086E990E00E945E0DC49886E990E00E94A4
:101380005E0DA7EDB0E00E940D0C0C94A509E2E003
:10139000F0E00E94ED0C0C949B09089581E080938D
:1013A00096010895A1E1B1E08C91082F033211F06C
:1013B0000C94E209A1E1B1E00E94B50C0E94C20CBC
:1013C0000C946F0AA1E1B1E08C91082F0B3111F060
:1013D0000C94F209A1E1B1E00E94B50C0E94C20C8C
:1013E0000C946F0AA1E1B1E0ECEBF0E22FEF91E099
:1013F0000E94A40DAFE9B1E00C9300919F01003071
:1014000018F011F00C94060A0C945B0AA1E1B1E00B
:10141000E8EFF0E22FEF91E00E94A40D002F0030E2
:1014200080E010F009F081E08F9340919F01A1E1ED
:10143000B1E0E8EFF0E22FEF91E00E94A40D002F61
:10144000041781E008F080E09F918923882311F43C
:101450000C94360AA1E1B1E00E94B50C0E94C20CC6
:101460000E94700A0C946F0A0C94590AE1E1F1E0B1
:1014700000919F01A1E5B1E00E944B10A1E5B1E010
:101480000E941310A8E9B1E00C930091980100307C
:1014900011F00C94510A0E94700A0C946F0A0C947B
:1014A000590AA1E1B1E00E94B50C0E94C20C0C9453
:1014B0006F0A0C946F0A00919801003011F00C949F
:1014C000670A0E94700A0C946F0A0C946F0AA1E1DB
:1014D000B1E00E94B50C0E94C20C0C946F0A0895F2
:1014E00081E08093A501A1E5B1E088278C93A1E973
:1014F000B1E088278C93ABE9B1E0E8EBF0E20E9421
:101500003C0F80E090E0A9E9B1E08D939C93A1E1CC
:10151000B1E00E945310082F0F93A1E1B1E0E0EA7F
:10152000F1E0222791E00E94A40D402F0F91041BAF
:10153000AFE9B1E00C93A1E1B1E00E945310EA2FB2
:10154000FB2F00919F013197E01BF10B0FEFA1E5FD
:10155000B1E00E944B10A1E9B1E088278C93A1E58E
:10156000B1E0E2EAF1E0222791E00E94A40DAFE9A8
:10157000B1E00C9300919F01003011F00C94C70A68
:10158000A1E5B1E00E945310AFE9B1E08C9381E096
:101590008093A40140919F010091A401041718F0C9
:1015A00011F00C94220B80E3482FA4EAB1E0AD9037
:1015B000BB24A0E5B1E0AA0DBB1D0C91041781E08E
:1015C00008F480E08F9389E3482FA4EAB1E0AD905E
:1015D000BB24A0E5B1E0AA0DBB1D0C91041781E06E
:1015E00010F009F080E09F918923882311F40C9476
:1015F0001A0BA4EAB1E0AD90BB24A0E5B1E0AA0DBE
:10160000BB1D8C91A5EAB1E0AD90BB24A0E9B1E08F
:10161000AA0DBB1D8C93A5EAB1E08C918F5F8C93D2
:1016200080E0A5EAB1E0AD90BB24A0E9B1E0AA0D4D
:10163000BB1D8C93A4EAB1E08C918F5F8C9310F466
:101640000C94CA0AA1E9B1E00E941310A9E9B1E023
:101650000D931C93A1E5B1E0E2EAF1E0222791E0CD
:101660000E94A40D002F003018F011F00C943A0BDA
:101670000C94410B8091B600877F8093B6000C9448
:10168000460B8091B60088608093B600A1E5B1E07A
:101690000E945310082F0F93A1E5B1E0E2EAF1E0B8
:1016A000222791E00E94A40D402F0F91041BAFE967
:1016B000B1E00C93A1E5B1E00E945310EA2FFB2F9B
:1016C00000919F013197E01BF10B0FEFA1E5B1E015
:1016D0000E944B10A1E5B1E00E94680EEDE0F0E041
:1016E000ABE9B1E00E944510A9E9B1E00D911C9170
:1016F000013050E0150711F00C949C0BA1E1B1E012
:10170000EAEFF0E20E94900DA1E1B1E00E946D0CC1
:10171000E7EBF0E00E94BD0FA1E1B1E00E946D0C8B
:10172000E2E0F1E20E94900DA1E1B1E00E94B50C6F
:101730000E94C20C0C940C0C023050E0150711F002
:101740000C94C00BA1E1B1E0E4E0F1E20E94900D45
:10175000A1E1B1E00E946D0CEBEBF0E00E94BD0F47
:10176000A1E1B1E00E946D0CE2E0F1E20E94900D77
:10177000A1E1B1E00E94B50C0E94C20C0C940C0CCB
:10178000033050E0150711F00C94DC0BA1E1B1E03F
:10179000ECE0F1E20E94900DA1E1B1E00E946D0C3D
:1017A000E6ECF0E20E94900DA1E1B1E00E94B50CE0
:1017B0000E94C20C0C940C0C063050E0150711F07E
:1017C0000C94000CA1E1B1E0E4E1F1E20E94900D83
:1017D000A1E1B1E00E946D0CEFEBF0E00E94C20FBE
:1017E000A1E1B1E00E946D0CE2E0F1E20E94900DF7
:1017F000A1E1B1E00E94B50C0E94C20C0C940C0C4B
:10180000A1E1B1E0ECE1F1E20E94900DA1E1B1E0D3
:101810000E94B50C0E94C20C08950D911D912D914E
:101820003C9181E0080F8827181F281F381F3C9320
:101830002E931E930E930895ED91FC91EF5FFF4F51
:10184000FC93EE930895ED91FC91E150F040FC93F0
:10185000EE93089500FC10D0089503D024D001F831
:10186000F9CF0024E89457FF02C009D0689400F82B
:101870000BD010F80124089502D009D00895509596
:1018800040954F5F5F4F0895E89417FF08950095C6
:1018900010950F5F1F4F6894089599231AF480954F
:1018A000909501960895352F242FE894452B11F437
:1018B00068940895512F402F0027112780E1440F8D
:1018C000551F001F111F021B130B416018F4020F5C
:1018D000131F4E7F8A9599F708958F938D918823D2
:1018E000E9F711978F910895A4E3B7E018D08830F5
:1018F00091F08D3039F03323C9F38D933A9563FE1F
:1019000044D0F4CF63FC04C08DE03FD08AE03DD0EA
:1019100088278C93089539D011973395E7CF0F928C
:101920009F93AF93BF937F9380918A008823E1F3C5
:10193000F89480918A008A9580938A00909188001B
:10194000A0E6B0E0A90F0024B01D8C9193959832C9
:1019500009F499279093880078947F91BF91AF9173
:101960009F910F900895A4E3B7E08D91882311F023
:101970000CD0FBCF08950E94640E802D11F005D08D
:10198000FACF08958DE001D08AE09F939FB79F938F
:10199000AF93BF930F937F939091B5009832E1F38B
:1019A000F8949091B50093959093B5009927009184
:1019B000B400ABE8B0E0A00FB91F8C9303950832D8
:1019C00009F400270093B400559A7F910F91BF91BD
:1019D000AF919F919FBF9F91089588EE93E06ED045
:1019E0003197D9F7089500FC05D0089530D005D07F
:1019F00001F8F9CF37D03FD00895842F952FA62F27
:101A0000B72FE894452B462B472B11F46894089583
:101A1000402F512F622F732F0027112722273327A2
:101A2000F0E2440F551F661F771F001F111F221F72
:101A3000331F081B190B2A0B3B0B416028F4080FBE
:101A4000191F2A1F3B1F4E7FFA9559F7089500244E
:101A5000E89477FF02C006D0689400F809D010F827
:101A60000124089512D04F5F5F4F6F4F7F4F08954D
:101A7000E89437FF089500951095209530950F5FF5
:101A80001F4F2F4F3F4F6894089540955095609594
:101A90007095089537FF089500951095209530951D
:101AA0000F5F1F4F2F4F3F4F08953197F1F7089564
:101AB000689462F80895E89462F80895EF93FF93AC
:101AC000EE27E82BE92B31F0E0EAFFE03197F1F760
:101AD0000197D1F7FF91EF9108950F921F922F92E6
:101AE000C801D901489F80014A9F90014B9F202C3B
:101AF000499F100D211D321D5A9F202C589F100DFB
:101B0000211D321D599F200D311D689F200D311D53
:101B1000699F300D789F300D2F901F900F90089582
:101B20000E94640E0D920020D9F70895369A3699D6
:101B3000FECF369A3699FECF84B195B1089599912A
:101B40000027A90FB01F1197492F4A955E2F6F2FBD
:101B5000E89411274395203019F0C895802D01C0D5
:101B600080818823B9F07C917723A1F0781739F42C
:101B70000EF0042F1395689411963196EBCF112334
:101B800021F0411BA11B1127B10BE894E52FF62F83
:101B90001196E0CF882311F0002708950895D19081
:101BA000E190F190019108952191319141915191EC
:101BB0000895102F90E8FF0C001F0927990FF79444
:101BC0001078652F90E8440F551F5927990F4795B6
:101BD000607800380895FF0C90E89027110F9795D2
:101BE000F794092F0895502F2D2D3E2D4F2D612F45
:101BF00008952DEC3CEC4CEC5DE366270FC0CFDF85
:101C0000F2DFDD24EE2490E8F92E0FE307C0CCDFED
:101C100005C02227332740E251E46627552351F1BE
:101C2000002381F1C6DF71F116270058505808943F
:101C3000050B18F407FD03C025C007FD23C046951A
:101C400037952795F694E794D79422D0FF202AF071
:101C5000DD0CEE1CFF1C015073F09D2D969548F095
:101C6000DD203AF4EE202AF491E0D90E9927E91EFE
:101C7000F91EB1CF07C09FE7092FF92A9FEFD92E90
:101C8000E92E0895DD24EE24FF240027112708956E
:101C90009F929924AA24BB2488E1D216E306F40675
:101CA00028F0D21AE30AF40A089401C08894991C17
:101CB000AA1CBB1CDD0CEE1CFF1C8A9571F7D92CED
:101CC000EA2CFB2C9F900895C8953196002008952A
:101CD0000E945B0DE89488278A938A93D3DF1127AB
:101CE0008D918032E9F31197BBD098F08D3229F4B1
:101CF000109511968C91B4D060F08E3229F4119623
:101D00008C91AED008F446C022960E94580D81E016
:101D100008958C91A5D0D8F547D01196D0F70395AA
:101D20008D919ED0E0F38E3229F48C9199D010F4ED
:101D30001196FBCF853419F0853609F055C0119600
:101D40008C918ED060F08D3219F08B3221F0DCCF87
:101D500008800094088211968C9182D0A8F6805356
:101D6000898311968C917CD058F49981990F990FA1
:101D70000980900D990F8053890F8983873220F64F
:101D80008981988199230AF48195080F2DC08E329C
:101D900089F611968C9164D068F606D018F01196E9
:101DA0000A95F8CF1196C1CF4F2D3E2D2D2DDD0C6C
:101DB000EE1CFF1CA8F0DD0CEE1CFF1C88F0D20E00
:101DC000E31EF41E68F0DD0CEE1CFF1C48F080538F
:101DD00009F06894D80E8827E81EF81E08F00895C8
:101DE000F42EE32ED22E089534D019F116F509837E
:101DF00008E921D00695882787959F2D9F77980F12
:101E0000F92E0150000F110F07958981882379F071
:101E10001AF48195898306C0ECDE89818A958983CD
:101E2000D9F705C0F6DE89818A958983D9F722968C
:101E3000089528DFFCCF0DD041F0FF2032F00A9545
:101E400031F0DD0CEE1CFF1CD2F788940895089445
:101E5000089500240D280E280F28002A0020089538
:101E6000803320F08A3310F40894089588940895FC
:101E700091E005C092E003C094E001C098E024DF47
:101E80000D929A95E1F708957F930F93AF93BF93C7
:101E90008F939F938FB78F93E89480918A0008E285
:101EA000081B21F49CB10E94580D13C000918900B9
:101EB000A0E6B0E077279CB1A00FB71F9C93689471
:101EC000839580938A000395083209F400270093D4
:101ED00089009D3011F40E94CE098F918FBF9F9190
:101EE0008F91BF91AF910F917F9118957F93AF9391
:101EF000BF938F939F938FB78F939091B500992342
:101F000099F09A959093B5009927ABE8B0E080914D
:101F1000B300A80FB91F9C918395883209F48827D4
:101F20008093B3009CB901C055988F918FBF9F914A
:101F30008F91BF91AF917F911895040F151F261FA8
:101F4000371F0895041B150B260B370B0895041734
:101F50001507260737070895000F111F221F331F8B
:101F6000089500951095209530950F5F1F4F2F4FC6
:101F70003F4F0895019110810EC00191119121915F
:101F800030810BC00191108117FF05C03FEF2FEF8B
:101F900004C0008111272227332737FF03C0E1DF68
:101FA0008DE28D93CF93DF93CF92DF92EF92AA24AD
:101FB000BB24CC24DD24EE2440E2CAE0DD2755E03A
:101FC00093E38881890F87FD9F7083FD907F891B34
:101FD00089935A95A9F7C0DFAA1CBB1CCC1CDD1C39
:101FE000EE1C4A9551F7E894EFE0FF2782910ED05E
:101FF000EB30E0F71EF068948A2D0CD088278D9383
:10200000EF90DF90CF90DF91CF910895982F829538
:1020100001D0892F8F70805D26F0803309F40895F8
:1020200068948D93089500271127222733271DD008
:102030008A3328F4803318F005D015D0F9CF0EF488
:1020400090CF089580538F93402F512F622F732F7D
:1020500083DF82DF72DF80DF8F919927080F191FDE
:10206000291F391F08958D910895E894FCDF80326F
:10207000E9F38B32D9F38930C9F38D3211F46894C6
:10208000F2CF089588278D93089594E081918D93E0
:102090009A95E1F7089581918D930A9519F0882317
:1020A000D1F70895EFCF8FEF83959D919923E1F7B5
:1020B0000895689463F80895000000003A003D0018
:1020C000323A31313D00574F463130330000323A19
:1020D000313D0000323A333D0000323A343D0000D9
:1020E000323A353D0000323A363D0000323A373D53
:1020F0000000323A383D00002A0023303A4144586B
:102100003D00210023303A4944473D0023303A49FD
:10211000444E3D0023303A4241543D0023303A457D
:1021200052523D5B53796E746178204572726F72C2
:042130005D2100002D
:00000001FF
